:020000040000FA
:020000000528D1
:08000800052883168E100E146A
:10001000831285010730990083160930850000306E
:100020008100831285100515FA30DE20FA30DE20BB
:10003000A501851D2D2805181928EB20051819285C
:1000400046206620251C1928742025182928CF2031
:10005000192802308506C42019280B30DE208519A6
:1000600019280B30DE2085191928B92005113F20E9
:100070006620251C37288F20B9200515192805185A
:100080003F28EB2005183F28000000002A3084009C
:100090002030A3005220240880000000840AA30B13
:1000A0004A280800A401EB20A40A03195C28051CB7
:1000B0005328EB20051C5328EB20A40A03196528BC
:1000C00005185C28EB2005185C28080025142A3048
:1000D00084000230A300840A0008003C031D73283A
:1000E000A30B6B28251008002A308400A0012030C3
:1000F000A3009C200008A2000230A2020530A90043
:100100002208210203198928A20AA90B8028251098
:100110008E28840AA00AA30B7928251408002A3007
:100120008400A0012030A3000008A100A420840ABC
:10013000A00AA30B94280800200883169B001C1417
:100140001A088312A1000800200883169B0083125E
:10015000210883169A001C1555309D00AA309D0079
:100160009C149C18B12883128C1383161C118312C3
:1001700008000A30A30005156430DE200511643044
:10018000DE20A30BBB2808000A30A3000511323083
:10019000DE2005153230DE20A30BC6280800033010
:1001A000A3000511FA30DE20FA30DE200515FA3002
:1001B000DE20FA30DE20A30BD1280800A600043090
:1001C000A7003130A800E428A80BE328A70BE128FA
:1001D000A60BDF2808000A30A600A60BED280800B1
:0207FE00B03415
:02400E0082012D
:00000001FF
